:100000008FC05CC0000055C000000000882391F044
:1000100006B306958A95D9F08A3049F09027813049
:1000200019F0069517950BC090FD75C008C000FD2E
:1000300072C005C0209719F0219709F4EE27109798
:1000400029F0119719F4B898BA98BB98189563D00D
:10005000312F00FF2CC0D0E0C0ECEE2319F43D336B
:1000600071F7222731932327E33048F311F43C3012
:10007000F0F4422D4C5FE41710F32223C1F4222048
:10008000B1F0432D31E1433179F04C3169F034E185
:10009000473151F0403241F038E1423229F04132EB
:1000A00019F03327493119F437BBB3E0A0ECEE2740
:1000B000C6CF882311F08A95439518950FB501FF97
:1000C00008C099279BBF8BE004E502BF04E008BF8E
:1000D000189502B711270A30141F9E01E8018823E2
:1000E00083E0E9F0021B130B083C20E01207B8F094
:1000F0000C3221E0120798F4169507950A9506BF71
:1001000002E00FBD04E009BF00E00BBF89E091E011
:1001100010E803E6DACF882740E44ABF4BBF1895C2
:1001200002E205BF01E003BF02E009BFAA27BB2727
:0E013000CC27DD27EE27FF27EEDF8895FECFD8
:02000004008278
:020000006AFF95
:02000004008476
:030000001E900748
:00000001FF
